:0200000480007A
:100000006F008004732F2034930F80006308FF0378
:10001000930F90006304FF03930FB0006300FF038E
:10002000130F000063040F0067000F00732F2034CC
:1000300063540F006F00400093E19153171F0000BD
:1000400023223FFC6FF09FFF732540F163100500F2
:10005000970200009382020173905230735000188F
:10006000970200009382020273905230B702008020
:100070009382F2FF7390023B9302F0017390023A75
:1000800097020000938282017390523073502030A7
:1000900073503030735040309301000097020000DD
:1000A000938282F673905230130510001315F501F8
:1000B000634C05000F00F00F930110009308D0056A
:1000C000130500007300000093020000638E02001D
:1000D00073905210B7B20000938292107390223046
:1000E00073232030E39A62F47350003097020000CB
:1000F0009382420173901234732540F173002030D3
:10010000930010001301000033972000930E10009D
:1001100093012000631ED7539300100013011000B9
:1001200033972000930E2000930130006312D753C1
:10013000930010001301700033972000930E000805
:10014000930140006316D751930010001301E000A3
:1001500033972000B74E000093015000631AD74F29
:10016000930010001301F00133972000B70E0080B8
:1001700093016000631ED74D9300F0FF1301000050
:1001800033972000930EF0FF930170006312D74D58
:100190009300F0FF1301100033972000930EE0FF4F
:1001A000930180006316D74B9300F0FF130170009A
:1001B00033972000930E00F893019000631AD749FB
:1001C0009300F0FF1301E00033972000B7CEFFFF4C
:1001D0009301A000631ED7479300F0FF1301F001C5
:1001E00033972000B70E00809301B0006312D74709
:1001F000B7202121938010121301000033972000B3
:10020000B72E2121938E1E129301C0006312D74591
:10021000B720212193801012130110003397200082
:10022000B74E4242938E2E249301D0006312D743DF
:10023000B720212193801012130170003397200002
:10024000B79E9090938E0E089301E0006312D74101
:10025000B7202121938010121301E0003397200072
:10026000B74E48489301F0006314D73FB7202121CF
:10027000938010121301F00133972000B70E008015
:10028000930100016316D73DB720212193801012FE
:10029000130100FC33972000B72E2121938E1E12EC
:1002A000930110016316D73BB720212193801012D0
:1002B000130110FC33972000B74E4242938E2E2438
:1002C000930120016316D739B720212193801012A2
:1002D000130170FC33972000B79E9090938E0E0808
:1002E000930130016316D737B72021219380101274
:1002F0001301E0FC33972000B74E484893014001BA
:100300006318D7359300100013017000B3902000DC
:10031000930E000893016001639CD033930010009A
:100320001301E00033912000B74E000093017001EB
:100330006310D13393003000B3901000930E80010E
:10034000930180016396D0311302000093001000E6
:1003500013017000339720001303070013021200EB
:1003600093022000E31452FE930E000893019001C3
:100370006310D32F13020000930010001301E0005C
:10038000339720001300000013030700130212002C
:1003900093022000E31252FEB74E00009301A00129
:1003A0006318D32B13020000930010001301F00117
:1003B0003397200013000000130000001303070010
:1003C0001302120093022000E31052FEB70E0080C9
:1003D0009301B001631ED3271302000093001000A5
:1003E00013017000339720001302120093022000C3
:1003F000E31652FE930E00089301C001631AD7253D
:1004000013020000930010001301E000130000002D
:10041000339720001302120093022000E31452FECF
:10042000B74E00009301D0016314D72313020000DC
:10043000930010001301F0011300000013000000EE
:10044000339720001302120093022000E31252FEA1
:10045000B70E00809301E001631CD71F1302000058
:100460009300100013000000130170003397200068
:100470001302120093022000E31452FE930E0008B0
:100480009301F0016316D71D1302000093001000C2
:10049000130000001301E000130000003397200058
:1004A0001302120093022000E31252FEB74E000026
:1004B00093010002631ED71913020000930010007D
:1004C00013000000130000001301F0013397200017
:1004D0001302120093022000E31252FEB70E0080B6
:1004E000930110026316D717130200001301700066
:1004F0009300100033972000130212009302200093
:10050000E31652FE930E0008930120026312D715E2
:10051000130200001301E00093001000130000001C
:10052000339720001302120093022000E31452FEBE
:10053000B74E000093013002631CD7111302000074
:100540001301F001930010001300000013000000DD
:10055000339720001302120093022000E31252FE90
:10056000B70E0080930140026314D70F13020000FE
:100570001301700013000000930010003397200057
:100580001302120093022000E31452FE930E00089F
:1005900093015002631ED70B130200001301E00009
:1005A0001300000093001000130000003397200098
:1005B0001302120093022000E31252FEB74E000015
:1005C000930160026316D709130200001301F001C2
:1005D0001300000013000000930010003397200068
:1005E0001302120093022000E31252FEB70E0080A5
:1005F00093017002631ED7059300F00033111000C1
:10060000930E0000930180026314D1059300000251
:1006100033910000930E000293019002631AD103FC
:10062000B3100000930E00009301A0026392D00368
:100630009300004037110000130101803390200027
:10064000930E00009301B0026314D00163103002D6
:100650000F00F00F638001009391110093E11100EE
:100660009308D00513850100730000000F00F00F00
:10067000930110009308D0051305000073000000DB
:10068000731000C000000000000000000000000027
:10069000000000000000000000000000000000005A
:1006A000000000000000000000000000000000004A
:0C06B0000000000000000000000000003E
:1010000000000000000000000000000000000000E0
:1010100000000000000000000000000000000000D0
:1010200000000000000000000000000000000000C0
:1010300000000000000000000000000000000000B0
:081040000000000000000000A8
:040000058000000077
:00000001FF
